:020000040000FA
:0600000000000EEF00F00D
:0400080004EF00F011
:080018000CEF00F005D861D8DF
:10002000A8D8D0D865D8FBD78E0EC16EE10E926EDF
:10003000DC0E936ED00E946E0F0E956E000E966EC3
:10004000880ED56E100E806E0DD883CF11F0136A16
:10005000080E146E156A020EF76E8A0EF66E20D820
:10006000166A12000A0E036E43D80306FDE184905F
:10007000020EF76E780EF66E08008482F5CF83FFCD
:10008000849236D88482F538836E849231D80B00FE
:10009000F552F3E11200210E036E0306FEE1120099
:1000A00084900800F55201E10B008482F5CF83FFB4
:1000B00084928482F538836E8492EDDF84800B0015
:1000C000F552F3E1120084908482EFCF83FF849293
:1000D0008482EF38836E8492DEDF8480EC50F4E11A
:1000E00012008088050603E1FA0E056E8098120062
:1000F000F2A4FED7F2CF02F0F29CF29ED6CF00F02F
:10010000D7CF01F0660E00269E0E012201C0D7FF58
:1001100000C0D6FF0250C00BF212F2941200020E81
:10012000F76E800EF66EBCDF00EE0FF0E86A063266
:10013000E8363009ED6EE9500708F8E100EE07F007
:10014000C00E076E106ABFDF1200126A8350046E81
:100150001118030B0BE0113002E3E89201D0E882A2
:100160000418030B02E1120601D0122A04C011F098
:1001700012001490149283A602D0148801D014980F
:1001800014A604D014B802D01E0E156E14B807D0F1
:10019000155204E114B402D01480148401D01494D4
:1001A00014B607D014A805D0155201E01482149497
:1001B000156A155201E0150614A802D0148601D064
:1001C0001496120014A010D0162A060E165C02E136
:1001D000010E166E020EF76E940EF66E61DF020EC1
:1001E000F76E9E0EF66E5CDF1650010809E114A052
:1001F00006D0020EF76EA80EF66E50EC00F038D85E
:100200001650020809E114A006D0020EF76EB20ED5
:10021000F66E50EC00F02DD8165003080CE114A037
:1002200006D0020EF76EBC0EF66E50EC00F022D82F
:1002300014A201D08072165004080CE114A006D05C
:10024000020EF76EC60EF66E50EC00F014D814A233
:1002500001D08074165005080AE177DF125013268A
:1002600013C006F08FEC00F014A201D0136A120044
:100270001200120012001200333228010C06000096
:1002800080425954453D20202000805075736820DD
:100290005042200080202020202020202000C0204C
:1002A00020202020202020008046726571206B488D
:1002B0007A00805065722020207573008050576D41
:1002C0006178207573008050576D696E20757300DA
:020000040030CA
:08000000FFFAF6FEFFFFFBFF13
:00000001FF
